:0A2284000001020203030404050533
:100C9200E4F513F512F511F510C20EC20BC20DC226
:100CA2000C122170120AA07E1A7F008E5C8F5D7575
:100CB200641A756512755A1A755B1C75621A75632A
:100CC2005175661A75677FEE54E07003020DD9758F
:100CD20014007515808E168F17C374A99FFF741A9E
:100CE2009ECF2402CF3400FEE48F0F8E0EF50DF559
:100CF2000CF50BF50AF509F508AF0FAE0EAD0DAC0C
:100D02000CAB0BAA0AA909A808C3120F325026E598
:100D120015250BF582E514350AF58374CDF0E50B44
:100D22002401F50BE4350AF50AE43509F509E43541
:100D320008F50880C4E4F50BF50AF509F508AF0FCC
:100D4200AE0EAD0DAC0CAB0BAA0AA909A808C312D2
:100D52000F325031AE0AAF0BE5172FF582E5163E82
:100D6200F583E0FDE5152FF582E5143EF583EDF000
:100D7200EF2401F50BE43EF50AE43509F509E43503
:100D820008F50880B985145C85155D74002480FF20
:100D9200741A34FFFEC3E5659FF565E5649EF5644C
:100DA200C3E55F9FF55FE55E9EF55EC3E5619FF576
:100DB20061E5609EF560C3E55B9FF55BE55A9EF5D4
:100DC2005AC3E5639FF563E5629EF562C3E5679FDB
:100DD200F567E5669EF566D2E843D82090E668E0BE
:100DE2004409F090E65CE0443DF0D2AFD288D28A6A
:100DF200C2A8C2AA43E808D2FB90E680E020E1053F
:100E0200D20F121F5890E680E054F7F0538EF8C2CA
:100E12000E300C05120676C20C300E291218FE5046
:100E220024C20E1220DB200B1690E682E030E7048B
:100E3200E020E1EF90E682E030E604E020E0E41218
:0A0E42001FB41219FE12131D80C721
:1006760090E6B9E070030207271470030207A4246A
:10068600FE700302082724FB70030207211470037F
:1006960002071B1460731460762405600302088643
:1006A6001222C2400302089290E6BBE024FE6022BA
:1006B60014603324FD601114602224067048E55C42
:1006C60090E6B3F0E55D8037E56490E6B3F0E56566
:1006D600802DE55E90E6B3F0E55F8023E56090E669
:1006E600B3F0E561801990E6BAE0FF121FE0AA06B2
:1006F600A9077B01EA494B600DEE90E6B3F0EF9057
:10070600E6B4F002089202088B12220A020892123C
:1007160022A9020892121D820208921221F80208EA
:10072600921222C4400302089290E6B8E0247F6049
:100736001514601924027063A20BE43325E0FFA2AE
:100746000DE4334F8041E490E740F0803F90E6BCF3
:10075600E0547EFF7E00E0D394807C0040047D015F
:1007660080027D00EC4EFEED4F2484F58274223E1D
:10077600F583E493FF3395E0FEEF24A1FFEE34E624
:100786008F82F583E0540190E740F0E4A3F090E611
:100796008AF090E68B7402F002089202088B12220D
:1007A600C6400302089290E6B8E024FE60162402D2
:1007B600600302089290E6BAE0B40105C20B020893
:1007C6009202088B90E6BAE0705590E6BCE0547E43
:1007D600FF7E00E0D394807C0040047D0180027D92
:1007E60000EC4EFEED4F2484F58274223EF583E440
:1007F60093FF3395E0FEEF24A1FFEE34E68F82F5FA
:1008060083E054FEF090E6BCE05480131313541FAB
:10081600FFE0540F2F90E683F0E04420F0806D80D7
:10082600641222C8506690E6B8E024FE60192402DD
:10083600705A90E6BAE0B40104D20B804F90E6BA43
:10084600E064026047803E90E6BCE0547EFF7E0096
:10085600E0D394807C0040047D0180027D00EC4E54
:10086600FEED4F2484F58274223EF583E493FF3334
:1008760095E0FEEF24A1FFEE34E68F82F583800833
:10088600120080500790E6A0E04401F090E6A0E058
:030896004480F0AB
:01089900223C
:030033000222BEE8
:0422BE0053D8EF32D0
:10217000758CE0758AC0E58954F04401F589758E47
:0821800003D28CD2A9D2AF22D8
:03005B0002089AFE
:10089A00C0E0C083C082C0D075D000C004C006C00A
:0108AA000746
:1008AB00AF91530780EF64806003020A9153917FED
:1008BB00300903020A8FE54E64047070D3E53E9451
:1008CB00C8E53D94005003020A8F0537E53725E054
:1008DB002472F582E43424F583E53DF0A3E53EF084
:1008EB00E53725E02470F582E43424F583E0FEA39C
:1008FB00E0FFD394C8EE9400402FEF25E0FFEE33DA
:10090B00FEEF2444FFEE34FDFEE53725E02472F5BF
:10091B0082E43424F583E0FCA3E0D39FEC9E4009F2
:10092B00752D01754E00753700020A89E54E64017D
:10093B0060030209EFD3E53E94C8E53D94005003F4
:10094B00020A8F0537E53725E02472F582E434245B
:10095B00F583E53DF0A3E53EF0E53725E02470F5A2
:10096B0082E43424F583E0FEA3E0FFD394C8EE9435
:10097B0000406EEF25E0FFEE33FEEF2444FFEE3434
:10098B00FDFEE53725E02472F582E43424F583E09F
:10099B00FCA3E0D39FEC9E4048054FE54F640270EB
:1009AB003DE53714F534752D01E53725E0246EF55B
:1009BB0082E43424F583E0FEA3E024C8F539E43E59
:1009CB00F538E53725E02470F582E43424F583E02F
:1009DB00FEA3E024C8F546E43EF545754E00753799
:1009EB0000020A89E54E64027061C3E53E94C8E5D6
:1009FB003D94004048D3E53E94C8E53D940040103B
:100A0B00D3E53E9546E53D95455005752D00802770
:100A1B00D3E53E9546E53D9545400FD3E53E9539EB
:100A2B00E53D95385004052D800DD3E53E9539E510
:100A3B003D95384008052D753D00753E00E52D654B
:100A4B002E7041F54EF53DF53E8039E54EB405343B
:100A5B00D3E53E9401E53D94004029E53725E0249C
:100A6B0072F582E43424F583E53DF0A3E53EF00511
:100A7B0037052DE52DB40F06754E00752D00753D10
:060A8B0000753E00C209E7
:0F0A9100D007D006D004D0D0D082D083D0E032AE
:101A00001201000200000040181633160000010207
:101A100000010A0600020000004001000902350032
:101A200001010080FA0904000005FF00000007051D
:101A30000102400000070582020002000705810242
:101A400040000007058602000200070508020002A8
:101A50000009022E0001010080FA0904000004FFC1
:101A60000000000705010240000007058202400057
:101A70000007050202000200070581024000000481
:101A800003090410035100480059002D004300438E
:101A90000044001603490043002D00310036003891
:0B1AA000003000330020002000000098
:10041900608025AC030A0101030401070000000202
:10042900000002000A2B0B13111515110000000022
:100439000000003F040A0103030401070000001043
:10044900020002000A2B0B130B1515110000000006
:100459000000003F04140201030401070000000228
:10046900000002000A2B0B131115111100000000E6
:100479000000003F04140103030401070000000009
:10048900020002000A2B0B130B15151100000000C6
:100499000000003F60242633000000000000000037
:1004A9000000000000000000000000000000000043
:1004B90000000000000000000000000047262C801A
:0604C900000009EA4E00EC
:1017890090E60174EAF090E6F574FFF090262CE0FB
:1017990090E6F3F090262DE090E6C3F090262EE037
:1017A90090E6C1F090262FE090E6C2F0902631E055
:1017B90090E6C0F0902632E090E6F4F075AF077439
:1017C90025F59A74ACF59B759DE4E4F59EFF90E6CA
:1017D9007BE090E67CF00FBF80F490E67174FFF037
:1017E900F5B490E672E04480F043B680000000E46E
:1017F90090E6C4F000000090E6C5F0902633E09032
:10180900E6C6F0902634E090E6C7F0902635E090E1
:10181900E6C8F0902636E090E6C9F0902637E090C9
:10182900E6CAF0902638E090E6CBF0902639E090B1
:0B183900E6CCF090263AE090E6CDF0FF
:011844002281
:030043000219009F
:030053000219008F
:10190000022188000221CE000221B8000221A0009D
:10191000021E5500021DE1000222CA000222CB0075
:101920000222CC000222CD00021F27000215E50092
:101930000222CE000222CF000222D0000222D100D9
:101940000222D2000222CB000222D3000222D400C3
:101950000222D5000222D6000222D7000222D8009D
:101960000222D9000222CB000222CB000222CB00AD
:101970000222DA000222DB000222DC000222DD0069
:101980000222DE000222DF000222E0000222E10049
:101990000222E2000222E3000222E4000222E50029
:1019A0000222E6000222E7000222E8000222E90009
:0819B0000222EA000222EB0012
:101FB40090E682E030E004E020E60B90E682E03038
:101FC400E119E030E71590E680E04401F07F147EEB
:0C1FD400001219B890E680E054FEF022E4
:1020DB0090E682E044C0F090E681F0438701000077
:0420EB0000000022CF
:101F5800300F0990E680E0440AF0800790E680E0C0
:101F68004408F07FDC7E051219B890E65D74FFF036
:0F1F780090E65FF05391EF90E680E054F7F0228F
:021FE000A9074F
:101FE200AE66AF678F828E83A3E064037017AD0184
:101FF20019ED7001228F828E83E07C002FFDEC3E72
:09200200FEAF0580DF7E007F00C7
:01200B0022B2
:1019B8008E1C8F1D90E600E054187012E51D24015E
:1019C800FFE4351CC313F51CEF13F51D801590E6D5
:1019D80000E05418FFBF100BE51D25E0F51DE51CC0
:1019E80033F51CE51D151DAE1C7002151C4E600557
:0619F8001220EF80EE2238
:1020EF007400F58690FDA57C05A3E582458370F904
:0120FF0022BE
:1004CF0060A5250518244242424242424224183E6A
:1004DF0008080808080808080E087E4204081020BB
:1004EF00204242423C1C2242404020182042423CC3
:1004FF007820207E222224242830201C22424040B3
:10050F00261A0202027E1824424242261A020224AE
:10051F0038080808080808101022227E3C42424280
:10052F002418244242423C1C244040586442424218
:10053F0024180000000000FE00000000001C3253D1
:10054F004D4141414141221CE7424242427E4242DB
:10055F004242E71C08080808081414222277E742D1
:10056F0042223C241414180808C1824225AA000014
:10057F004224F200004224F40000412410004124E0
:10058F0011004124FB0002321040C107C104014B8E
:10059F0000012500442501000000004424F700005D
:1005AF000000013C004124F600608024720000002E
:1005BF00000000000000000000000000000000002C
:1005CF00000000000000000000000000000000001C
:1005DF00000000000000000000000000000000000C
:1005EF0000000000000000000000000000000000FC
:1005FF0000000000000000000000000000000000EC
:10060F0000000000000000000000000000000000DB
:10061F0000000000000000000000000000000000CB
:10062F000000000000000000000000000001370083
:10063F00014E01012EFF012D00023D00000134008B
:10064F00014F000238000002450000014D00025426
:10065F0000000235C350012C19C189013100C101BD
:06066F00014100013F0003
:101F87008E188F199024527403F0E4A3F07A247BFF
:101F9700527D027F411221399024527401F0A3E54A
:0D1FA70019F07A247B527D027F410221391E
:0B226E00C2B6C2B48FB1D2B4D2B62207
:0B227900D2B6C2B48FB1D2B4D2B622EC
:04215500AE05AD071F
:10215900E4FCE4FBAF05122279AF061222790BBB2E
:0621690060F20CBC40EC2A
:01216F00224D
:10203700AE05AD077F1512226EAF0612226E7F5FC7
:1020470012226E7F7512226EAF0512226E7F3F122B
:0A205700226E7F2512227902227901
:041BBF007B067F31F1
:021BC300AE036F
:101BC500EDC454F0F518EE75F008A4F519BF2D0411
:101BD5007A0A8020BF51047A0B8019BF48047A0C19
:101BE5008012BF59047A0D800BBF41047A0E800420
:101BF500EF24D0FAE4FBEA75F00BA42405F582E4A2
:101C05003425F583E5822BF582E43583F583E0F908
:101C1500E4FCE930E70DE51824022BFFE5192CFD5E
:0F1C2500122037E925E0F90CBC08E70BBB0BC711
:011C3400228D
:1018DF00C2B77FC87E001215CED2B77FAE12226E6E
:0F18EF007FA012226E7F6012226E7FAF02226EE8
:101845001218DFE4FDFF1221557B097D027F51123D
:101855001BC37B087D027F48121BC37B077D027F6C
:1018650059121BC37D02121BBF7B057D027F3612F9
:101875001BC37B047D027F38121BC37B037D027F64
:1018850030121BC37B027D027F33121BC37B017D9C
:10189500027F41121BC37B097D017F31121BC37B74
:1018A500087D017F36121BC37B077D017F2D121B2F
:1018B500C37D01121BBF7B057D017F32121BC37BDC
:1018C500047D017F2D121BC37B037D017F31121B1C
:0A18D500C37B027D017F36021BC3B6
:100AA00090E600E054E74410F000000000000090E1
:100AB000E61074A0F000000090E60B7401F090E6E0
:100AC0001274E0F0000000E490E613F000000090E3
:100AD000E61474E2F000000090E61574A0F0000047
:100AE0000090E6D27402F090E6047480F0000000FA
:100AF0007402F00000007406F00000007408F000BA
:100B00000000E4F000000012178990E6187408F065
:100B100000000090E619F000000090E61AF00000D6
:100B20000090E61BF0000000E490E671F075B47FE1
:100B300075A07F90E672F075B6FF75B1FF90E67014
:100B4000F075B2FF75B5FFC28CD2B01222B990E633
:100B50001074A0F000000090E611F000000090E694
:100B60005EE04408F0000000E490E68DF000000034
:100B700090E65EE04404F0000000E490E7C0F090EE
:100B8000E7C4F0A3F0A3F0A3F090E7F0F090E68FB5
:100B90007440F000000090E65EE04440F000000089
:100BA0007E027F0090F800E4F0A3DFFCDEFA90E61E
:100BB000987402F0000000E490E699F00000007ED6
:100BC000027F0090F800E4F0A3DFFCDEFA90E65E1E
:100BD000E04480F0000000E490E69CF0000000900B
:100BE000E69DF00000007F9AFE12228E75270075A8
:100BF00028B47550017551907532107533B875521F
:100C00000675532C1222B190E67AE054FEF0E4FD12
:100C10007F9012221C7F647E001219B87DFF7F42F4
:100C200012221C7F647E001219B87D827F4E122230
:100C30001C7540FF43A020E4F54490E782E540F0B6
:100C400090E781E544F01222B9D209754E0175355D
:100C500027753610752C0A121B377FD07E071215A8
:100C6000CE121B377FB87E0B1215CE121B377FA01A
:100C70007E0F1215CEC201C2B2D2F9C2F8E4F54B12
:100C800090E7C0E54BF043A01053917F53A0F002D2
:020C9000184505
:0E226000EF2401FBE43EFA7D047F4802211DBD
:10206100E544C313FFC374809F9025ABF0E4940053
:102071009025AAF0E544D3940040067540FF43A0A3
:0920810020E544700353A0DF22A6
:10141900E4FC9024FDE0FEA3E02400FDEC3EFC90FA
:101429002410E0FEA3E07A002400FFEA3EFEC3EDAB
:101439009FFFEC9EFE9024F2F0A3EFF09024F5E0DC
:101449002FF09024F4E03EF0D3EF9450EE648094B2
:10145900805011C39024F3E094B09024F2E06480AA
:10146900947F50209024F2E0FEA3E0FF7C007D05EC
:10147900120E9B9025AAEEF0A3EFF0E49024F4F06D
:10148900A3F080339024F5E025E0FF9024F4E033C5
:10149900FE7C007D0A120EADAA06AB079024F2E08D
:1014A900FEA3E0FF7C007D05120E9BEF2BFFEE3AB9
:1014B9009025AAF0A3EFF0D39025ABE094FF9025F7
:1014C900AAE0648094804006E4F0A374FFF0C3901E
:1014D90025AAE0648094805004E4F0A3F09025AA42
:1014E900E0FEA3E0FF7C007D02120EADC3747F9F76
:0714F900F0E49E9025AAF02B
:0115000022C8
:101CA8007E247FFC1222609024FDE090E7C1F09032
:101CB80024FEE090E7C2F09025ABE090E7C3F090F7
:101CC80024FBE0600B43A0207540FF121419800329
:101CD800122061902452E540F07A247B527D017FE6
:101CE800211221399024527402F0A37480F07A24CE
:101CF8007B527D027F28122139E4902452F09025EE
:101D0800ABE0902453F07A247B527D027F28022195
:011D18003991
:10131D000555E55570020554054DB5360DE554B529
:10132D003508121CA8E4F554F55590E7C8E54EF0C4
:10133D00A3E52DF0A3E534F0E54D652C7024E54EC5
:10134D00601414600C14600924FD60050470108095
:10135D00001222508009E4FFFE121F8753A0EFE414
:10136D00F54D200003021418754B0190E7C0E54BB5
:10137D00F0E5A030E7032007F87FAE12226E90F063
:10138D000074AAF0A37411F0A374CCF0A374EEF062
:10139D00E490E690F090E6917405F0120FB790F09E
:1013AD000074AAF0A37411F0A374CCF0A374EEF042
:1013BD00E490E690F090E6917405F07FAF12226E06
:1013CD00C200E4F54B90E7C0E54BF09024F6E0B495
:1013DD000107E53C7003021B37121B377FD07E07D8
:1013ED001215CE121B377FD07E071215CE121B376A
:1013FD007FD07E071215CE121B377FD07E071215B8
:0C140D00CE121B377FD07E071215CE22B6
:0218FE00D322F3
:0219FE00D322F2
:0222C200D32225
:101D820090E680E030E73A00000090E6207402F02E
:101D9200000000E490E621F000000090E6247402C6
:101DA200F0000000E490E625F000000090E62674C2
:101DB20002F0000000E490E627F0000000D202806A
:101DC20016000000E490E620F000000090E6217486
:0F1DD20040F0000000C20290E6BAE0F54CD322C8
:1021F80090E740E54CF0E490E68AF090E68B04F036
:02220800D322DF
:0822A90090E6BAE0F526D3220D
:10220A0090E740E526F0E490E68AF090E68B04F049
:02221A00D322CD
:0222C400D32223
:0222C600D32221
:0222C800D3221F
:10008000E4FFF518F51990E6B9E0244B605224F32B
:10009000700302029924F870030202E124FA70034B
:1000A000020323241D6003020415E490E68AF09005
:1000B000E68BF090E6A0E020E1F990E68BE0E4F535
:1000C000B390E60174CAF0D20000000090E6047418
:1000D00080F00000007402F0000000E4F002041759
:1000E000E490E68AF090E68BF090E6A0E020E1F95B
:1000F00090E68BE0D3943F4024E4F5187440251833
:10010000F582E434E7F583E0FF74122518F582E404
:100110003424F583EFF00518E518B440DF7F8A7EBC
:100120000012228E902412E0FF7E0012229790246B
:1001300013E075F004A4FFAEF01222A0902417E0A3
:10014000C394025013902433E090E6C07005744EBF
:10015000F08016749CF08011902433E090E6C0701B
:1001600005749FF08003749DF0902435E024FF9285
:1001700006902432E024FF9205902436E024FF927A
:1001800008902440E0754200F543A3E0FEA3E07C24
:10019000002400F524EC3EF523902445E09024F65D
:1001A000F0902418E0F53AE53A7003753A0190248E
:1001B0001DE0FEA3E07C002400F528EC3EF527A31B
:1001C000E0FEA3E02400F551EC3EF550902419E048
:1001D000FEA3E02400F533EC3EF532A3E0FEA3E0FD
:1001E0002400F553EC3EF55290244DE0FFE4FDFE73
:1001F000FBFAF97801120EE3A804A905AA06AB07D9
:10020000902423E0FEA3E07C002400FFEC3EFEE40B
:10021000FDEB2FFFEA3EFEED39FDEC38FCC004C0DB
:1002200005C006C00790244EE0FFE4FCFDFEFBFA8B
:100230007901F8120EE3D003D002D001D000EF2BE9
:10024000F54AEE3AF549ED39F548EC38F547902492
:1002500021E0FEA3E07C002400F530EC3EF52F9079
:100260002447E0540FF53CE4FD7F9012221C9024BB
:1002700013E0FCA3E0FDA3E0FEA3E0FF9025011244
:100280000F56902501A3E0FDA3E0FEA3E0FFE4FCF0
:10029000902501120F5602041790E740740CF0A34A
:1002A0007410F0A3740CF0A37426F0A37407F0A3E9
:1002B00074EEF0A37401F0A37403F0A37453F03050
:1002C0000205E4A3F0800690E74974FFF000000007
:1002D000E490E68AF000000090E68B740AF00204D5
:1002E0001790E6BCE0902657F07A267B577D017F79
:1002F000501221397A267B577D017F501221399087
:10030000E6BEE0FD7AE77B407F5012211DE490E6D7
:100310008AF000000090E6BEE090E68BF00000005E
:10032000020417E490E68AF090E68BF090E6A0E0F5
:1003300020E1F990E68BE0F518C29890E740E0C321
:1003400094304014E534242FFFE433FEE0D39FEED5
:100350006480F8748098401190E740E0F4600302F4
:1003600003ECE54E60030203EC43A01090E740E08D
:10037000F4600AE0B4300EE52D64016008D209751E
:100380004E0402041790E740E0C394315003020486
:1003900017E534242FFFE433FEE0D39FEE6480F8AA
:1003A0007480985072E024D1F52E652D6069E0B418
:1003B0000A03752E6190E740E0B40B03752E62903E
:1003C000E740E0B40C03752E6390E740E0B40D0302
:1003D000752E6490E740E0B40E03752E6590E740FB
:1003E000E0B40F03752E66754E02802B90E740E057
:1003F000B4200CE54E700843A010754E058018908F
:10040000E740E0B41104D201800D90E740E0B4125F
:0804100006C2018002D322C3E1
:0104180022C1
:10218800C0E0C083C082D20C5391EF90E65D740129
:08219800F0D082D083D0E032C8
:1021B800C0E0C083C0825391EF90E65D7404F0D014
:0621C80082D083D0E0325A
:1021CE00C0E0C083C0825391EF90E65D7402F0D000
:0621DE0082D083D0E03244
:101E5500C0E0C083C08285625E85635F855F8285E1
:101E65005E83A37402F0855A60855B618561828516
:101E75006083A37407F05391EF90E65D7410F0D082
:061E850082D083D0E032A0
:1021A000C0E0C083C082D20E5391EF90E65D740808
:0821B000F0D082D083D0E032B0
:101DE100C0E0C083C08290E680E030E720855A5E83
:101DF100855B5F855F82855E83A37402F085626087
:101E0100856361856182856083A37407F05391EFD7
:0D1E110090E65D7420F0D082D083D0E032E6
:0122CA0032E1
:0122CB0032E0
:0122CC0032DF
:0122CD0032DE
:101F2700C0E0C083C08290E65EE054FBF000000092
:101F370090E68F7440F00000005391EF90E65FE069
:101F47004404F090E65EE04404F0D082D083D0E011
:011F57003257
:1015E500C0E0C0F0C083C082C0D075D000C000C0CC
:0D15F50001C002C003C004C005C006C0074D
:1016020090E65EE054F7F090E6A1E020E1F990E781
:1016120080E0FF14601614602624D0603A243460FF
:1016220059146060147062752200805D90E782E058
:10163200F54090E781E0F5449024FBE4F0804A9085
:10164200E782E0902410F090E781E0902411F0907E
:1016520024FB7401F0803290E781E07005121B37A1
:10166200802790E781E0B40105122240801B90E7B9
:1016720081E0B403141220B3800F90E781E024FFCD
:1016820092078005752200D20300000090E68DE4E7
:10169200F05391EF90E65FE04408F090E65EE0449C
:0216A20008F04E
:1016A400D007D006D005D004D003D002D001D0009A
:0B16B400D0D0D082D083D0F0D0E03244
:0122CE0032DD
:0122CF0032DC
:0122D00032DB
:0122D10032DA
:0122D20032D9
:0122D30032D8
:0122D40032D7
:0122D50032D6
:0122D60032D5
:0122D70032D4
:0122D80032D3
:0122D90032D2
:0122DA0032D1
:0122DB0032D0
:0122DC0032CF
:0122DD0032CE
:0122DE0032CD
:0122DF0032CC
:0122E00032CB
:0122E10032CA
:0122E20032C9
:0122E30032C8
:0122E40032C7
:0122E50032C6
:0122E60032C5
:0122E70032C4
:0122E80032C3
:0122E90032C2
:0122EA0032C1
:0122EB0032C0
:0616BF008F1A8C1B8D1C2C
:1016C500531A0753B0F77F0A7E001215CEE4F51DB5
:1016D500F51EC37402951EFFE51AA807088002C30C
:1016E50013D8FC30E00543800280035380FD7F0A58
:1016F5007E001215CE4380017F0A7E001215CE535F
:1017050080FE7F0A7E001215CE051EE51E700205BD
:101715001DC39403E51D6480948040B6E4F51DF572
:101725001EC37409951EFFE51CAE1BA8070880059E
:10173500CEC313CE13D8F930E0054380028003539E
:1017450080FD7F0A7E001215CE4380017F0A7E0050
:101755001215CE5380FE7F0A7E001215CE051EE5BA
:101765001E7002051DC3940AE51D6480948040B176
:1017750043B0087F0A7E001215CE53B0F77F0A7E6C
:04178500000215CE7B
:09228E00AD07AC06E4FF0216BF27
:09229700AD07AC067F040216BF7E
:0922A000AD07AC067F010216BF78
:10221C00902452EDF0EFC313FF7A247B527D010220
:02222C00213956
:1015010053A0F043A0067FEE7E021215CE53A0F049
:1015110043A0027FEE7E021215CE53A0F043A0033A
:101521007FEE7E021215CE53A0F043A0017FEE7E26
:10153100021215CE53A0F043A0097FEE7E021215D0
:10154100CE53A0F043A0087FEE7E021215CE53A029
:10155100F043A00C7FEE7E021215CE53A0F043A003
:10156100047FEE7E021215CE53A0F043A0067FEE5B
:101571007E021215CE53A0F043A0027FEE7E02122E
:1015810015CE53A0F043A0037FEE7E021215CE5379
:10159100A0F043A0017FEE7E021215CE53A0F043CE
:1015A100A0097FEE7E021215CE53A0F043A0087F62
:1015B100EE7E021215CE53A0F043A00C7FEE7E0208
:0D15C1001215CE53A0F043A0047FEE7E0271
:1015CE00EF7803C333CE33CED8F9FFEF4E6007EF7B
:0715DE001F70F81E80F522CA
:0522B900D283D2842253
:10210000C2837F127E001215CEC284D2837F127EDC
:0D211000001215CED2847F127E000215CE83
:10222E00E4FDFC1221000DBD00010CBC10F5BD201B
:01223E00F2AD
:01223F00227C
:10110C00902501E0FCA3E0FDA3E0FEA3E0FF90240A
:10111C00F7120F56300502C2B09024F6E07006129A
:10112C00224043A0403006030211FA752201E47FED
:10113C00E87E03FDFC9024F7E0F8A3E0F9A3E0FAC5
:10114C00A3E0FBC3120F3250030211E8E522640145
:10115C0060030211E87FDD7E031219B8121CA890FF
:10116C0024F7E0FCA3E0FDA3E0FEA3E02418FFEECF
:10117C0034FCFEED34FFFDEC34FFFC9024F7120F31
:10118C00569024F7E0FCA3A3A3E4FFFEFDEC781833
:10119C00120F4390E7C4EFF09024F7A3E0FDA3A354
:1011AC00E4FFFEE4FC7810120F4390E7C5EFF090DB
:1011BC0024F7A3A3E0FEA3E4FFE4FDFC7808120FE0
:1011CC004390E7C6EFF09024F7E0FCA3E0FDA3E02A
:1011DC00FEA3E0FF90E7C7EFF002113AE522B4015D
:1011EC00169024F9E0FEA3E0FF1219B880097522CD
:1011FC0001E522640160FA9024F6E0700653A0BF6A
:09120C001220B3300502D2B02219
:101C35008F1F8E1E8D1D8C1CE4FFFEFDFCAB1FAAA5
:101C45001EA91DA81CD3120F324057000000E4FF47
:101C5500FEFDE51CFC7818120F4390E6CEEFF00070
:101C65000000E4FFFEE51DFDE4FC7810120F439033
:101C7500E6CFEFF0000000E4FFE51EFEE4FDFC7892
:101C850008120F4390E6D0EFF0000000E51FFF902B
:101C9500E6D1EFF000000075BB04000000E5BB30A5
:031CA500E7FB2238
:081E1E008C1C8D1DAB07AA0608
:101E2600E4FDFCC3ED951DEC951C5022EA90E6D02E
:101E3600F0000000EB90E6D1F000000075BB050055
:0E1E46000000E5BB30E7FB0DBD00010C80D5B0
:011E5400226B
:10208A00AD07AC06000000ED25E0EC3390E6D0F099
:10209A00000000ED25E090E6D1F000000075BB04D9
:0920AA00000000E5BB30E7FB2259
:1021E400200102C2B230010BD2B27FE87E03121585
:0421F400CEC2B22283
:100FB700C20353A0F043A0091215CA53A0F043A0DF
:100FC700011215CA53A0F043A0031215CA53A0F08B
:100FD70043A0027FF47E011215CE53A0F043A00672
:100FE7007FF47E011215CE53A0F043A0047FF47E58
:100FF700011215CE53A0F043A00C7FF47E01121509
:10100700CE53A0F043A0087FF47E011215CE9024A2
:10101700F6E064017024E53C702053A0F043A0047F
:101027007FF47E011215CE53A0F043A00C7FF47E0F
:10103700011215CE53A0F043A0081221E412222E6C
:10104700754B0290E7C0E54BF012110C754B0390FE
:10105700E7C0E54BF030030302110BE4F51AF51B6B
:10106700C3E51B9528E51A9527500D122100051B8E
:10107700E51B7002051A80E8D3E5439400E5429426
:1010870000400BAD43AC42AF33AE32121E1ED3E568
:10109700249400E52394004007AF24AE2312208A4E
:1010A700E4F518F519C3E5199553E5189552502C31
:1010B70012200CE4F51AF51BC3E51B953A7480F86A
:1010C700651A98500D122100051BE51B7002051AC1
:1010D70080E60519E5197002051880C9E4F51AF5C7
:1010E7001BC3E51B9551E51A9550500D12210005BC
:1010F7001BE51B7002051A80E8AF4AAE49AD48AC44
:0411070047121C353A
:01110B0022C1
:10200C00000000E53325E0E5323390E6D0F0000027
:10201C0000E53325E090E6D1F000000075BB04002C
:0B202C000000E5BB20E7033003F822B2
:101B370053A0F043A0091215CA53A0F043A0011205
:101B470015CA53A0F043A0031215CA53A0F043A02F
:101B5700021215CA53A0F043A0061215BD53A0F0F8
:101B670043A00C1215CA53A0F043A0081215CA537C
:101B7700A0F043A0091215CA53A0F043A001121503
:101B8700CA53A0F043A0031215CA53A0F043A00202
:101B97001215CA53A0F043A0061215BD53A0F04377
:101BA700A00C1215CA53A0F043A0081215CAE4F5F9
:081BB7002590E7CBE525F022A3
:1020B30012150153A0F043A0061215CA53A0F04312
:1020C300A0021215CA53A0F043A0031215CA752526
:0820D3000390E7CBE525F022A4
:102240001215B712150175250190E7CBE525F0228F
:101D19000531E531B40803E4F531E53170057F0893
:101D2900FE804BE531B401067F0A7E008040E53133
:101D3900B402067F027E008035E531B403067F03D5
:101D49007E00802AE531B404067F017E00801FE50C
:101D590031B405067F057E008014E531B406067F9F
:101D6900047E008009E531B4070E7F0C7E00121F46
:091D7900877F467E001215CE2280
:10225000E54E600B053EE53E7002053D121D19225C
:0822B100E4F56DD2E9D2AF2281
:101E8B0090E678E020E6F9C2E990E678E04480F04D
:101E9B00EF25E090E679F090E678E030E0F990E617
:101EAB0078E04440F090E678E020E6F990E678E0C0
:061EBB0030E1D6D2E9225D
:101EF500A90790E678E020E6F9E56D702390E6788D
:101F0500E04480F0E925E090E679F08D68AF03A91B
:101F1500077569018A6A896BE4F56C756D01D322D1
:021F2500C322D5
:101EC100A90790E678E020E6F9E56D702590E678BF
:101ED100E04480F0E925E0440190E679F08D68AFB7
:101EE10003A9077569018A6A896BE4F56C756D034D
:041EF100D322C32213
:03004B0002121589
:10121500C0E0C083C082C085C084C086758600C01A
:10122500D075D000C000C001C002C003C006C00711
:1012350090E678E030E206756D060212FF90E678DA
:10124500E020E10CE56D64026006756D070212FF92
:10125500E56D24FE605F14603624FE70030212F013
:1012650024FC70030212FC240860030212FFAB6920
:10127500AA6AA96BAF6C056C8F82758300120E4C40
:1012850090E679F0E56C65687070756D05806B901A
:10129500E679E0AB69AA6AA96BAE6C8E82758300AC
:1012A500120E79756D02E5686401704E90E678E07E
:1012B5004420F08045E56824FEB56C0790E678E0AB
:1012C5004420F0E56814B56C0A90E678E04440F0F7
:1012D500756D0090E679E0AB69AA6AA96BAE6C8E74
:1012E50082758300120E79056C800F90E678E044D4
:1012F50040F0756D008003756D005391DFD007D008
:1013050006D003D002D001D000D0D0D086D084D072
:0813150085D082D083D0E032C4
:10211D00121EC1E56D24FA600E146006240770F3DB
:0C212D00D322E4F56DD322E4F56DD3223B
:10213900121EF5E56D24FA600E146006240770F38B
:0C214900D322E4F56DD322E4F56DD3221F
:03000000021AAB36
:0C1AAB00787FE4F6D8FD75816D021AF218
:100E4C00BB010CE58229F582E5833AF583E022505B
:100E5C0006E92582F8E622BBFE06E92582F8E222A5
:0D0E6C00E58229F582E5833AF583E49322BF
:100E7900F8BB010DE58229F582E5833AF583E8F0AF
:100E8900225006E92582C8F622BBFE05E92582C85B
:020E9900F22243
:100E9B00EF8DF0A4A8F0CF8CF0A428CE8DF0A42E6B
:020EAB00FE2225
:100EAD00C2D5EC30E709B2D5E4C39DFDE49CFCEE60
:100EBD0030E715B2D5E4C39FFFE49EFE120F62C367
:100ECD00E49DFDE49CFC8003120F6230D507C3E462
:060EDD009FFFE49EFE22CF
:100EE300E88FF0A4CC8BF0A42CFCE98EF0A42CFCAE
:100EF3008AF0EDA42CFCEA8EF0A4CDA8F08BF0A42C
:100F03002DCC3825F0FDE98FF0A42CCD35F0FCEB8A
:100F13008EF0A4FEA9F0EB8FF0A4CFC5F02ECD394F
:0F0F2300FEE43CFCEAA42DCE35F0FDE43CFC22BC
:100F3200EB9FF5F0EA9E42F0E99D42F0E89C45F015
:010F4200228C
:100F4300E8600FECC313FCED13FDEE13FEEF13FF8C
:030F5300D8F122B0
:0C0F5600ECF0A3EDF0A3EEF0A3EFF0220E
:101AB700020C92E493A3F8E493A34003F68001F2A7
:101AC70008DFF48029E493A3F85407240CC8C33330
:101AD700C4540F4420C8834004F456800146F6DFFF
:101AE700E4800B0102040810204080900419E47E72
:101AF700019360BCA3FF543F30E509541FFEE493F4
:101B0700A360010ECF54C025E060A840B8E493A3BA
:101B1700FAE493A3F8E493A3C8C582C8CAC583CAE5
:101B2700F0A3C8C582C8CAC583CADFE9DEE780BE9D
:010675000084
:100F6200BC000BBE0029EF8DF084FFADF022E4CC73
:100F7200F875F008EF2FFFEE33FEEC33FCEE9DEC3C
:100F8200984005FCEE9DFE0FD5F0E9E4CEFD22ED82
:100F9200F8F5F0EE8420D21CFEADF075F008EF2FCC
:100FA200FFED33FD4007985006D5F0F222C398FDBD
:050FB2000FD5F0EA225A
:00000001FF
